:10000000FF23831690000430850000308312A60081
:100010000430B2002608213E840080308000A60A09
:10002000B20B0A280030AB000030A0005F10003097
:10003000AC000030A5000030A7000030A800003060
:10004000AD0085160030A6000030A900A00A0030DF
:100050008A001F3020052D3E82004D289528A728B4
:10006000A728A728A728A728A728A728A728A72818
:10007000A728A728A728A728A728A728A7289C2813
:10008000F228F228F228F228F228F228F228F228A0
:10009000F228F228F228F228F228200EB200320CC0
:1000A0000339A6002608213E84000008AD00AD1DDE
:1000B000762800308A0026085E3E82006228652885
:1000C00068286B28251805146E28A51885146E2835
:1000D000251905156E28A51905166E28AD110D30C8
:1000E000FF3E031D70287428000094283030050559
:1000F000B00000308A0026087E3E820082288528D3
:1001000088288B28251830148E28A518B0148E281E
:10011000251930158E28A51930168E280D30FF3E72
:10012000031D8F2830088500FE2864001430FF3E30
:10013000031D97280000FE28640005108510051196
:1001400005121330FF3E031DA2280000FE28AD0A51
:1001500000308A002608AD3E8200B128C028CF2892
:10016000DE280430B200AD0303190510B728B82803
:100170000000AD0303190510BD28B20BB328ED280C
:100180000430B200AD0303198510C628C72800004B
:10019000AD0303198510CC28B20BC228ED2804301A
:1001A000B200AD0303190511D528D6280000AD0310
:1001B00003190511DB28B20BD128ED280430B20059
:1001C000AD0303190512E428E5280000AD03031967
:1001D0000512EA28B20BE028ED28AD03AD11F02896
:1001E000F128FE285F18FA281330FF3E031DF5287A
:1001F0000000FC285F107B210000FE2801308A00EF
:1002000083122908043E8200422971297129472955
:100210004C29712947294C29712947294C297129D1
:1002200047294C29712947294C29712947294C29EB
:10023000712947294C29712947294C29712971298C
:100240007129512971295729712971295C2962293C
:1002500071295C29622971295C29622971295C292B
:10026000622971295C29622971295C296229712915
:100270005C29622971295C297129712967297129F1
:100280006C297129051EA90A452900007529A90AAA
:10029000AB0CAB134B297529A90A051AAB175029CA
:1002A00075290030A9002B08AA005F147529A90A36
:1002B00085125A2900007529A90A85122B1885165E
:1002C00000007529A90AAB0CAB1366297529A90A88
:1002D00085166A29000075290030A9006F290000E1
:1002E0007529A90A7329742975290630FF3E031D53
:1002F00076297A29262801308A002C08803E82003F
:100300008329BA2AD52A01308A002A0EB400B40CF7
:10031000340C03398C3E82009029A129BA29DB29AB
:1003200003302A05B1003108213E84002A0DB300B4
:10033000330DF03980000930FF3E031D9C29000079
:10034000B92A03302A05B1003108213E8400000893
:10035000F039B4002A0CB500350C0F393404B30061
:100360003108213E8400330880000730FF3E031D22
:10037000B629B92A03302A05B1002A0CB400340C7E
:100380000739AF00AA1AC629C529C9292F09013E74
:10039000AF003108213E840000082F07B400310867
:1003A000213E8400340880000530FF3E031DD5291E
:1003B000D9290000B92A01308A002A0CB400B40CF3
:1003C000340C0739E43E8200EC29F629092A292A4F
:1003D0004B2A4B2A4B2A512A2A08AE000130AC0086
:1003E0000730FF3E031DF129F529B82A03302A05FD
:1003F000B10031083023B1002A1D012A3108A504BB
:10040000042AFF303106A5050330FF3E031D052AEF
:10041000B82A03302A05B1002A191A2A0230FF3EF1
:10042000031D0F2A132A00003108213E8400000812
:10043000AB00212A0030AB00310830232505031D15
:10044000AB0A1F30A9000530FF3E031D242A00001F
:10045000B82A02308A0007302A052F3E8200372A48
:100460003C2A402A402A402A402A402A402A25087D
:10047000AB001F30A900432A0230AC003F2A432AB8
:10048000412A422A432A0430FF3E8312031D442A94
:10049000492A0000B82A0830FF3E031D4C2A502A82
:1004A000B82A02308A0007302A05573E82005F2AA8
:1004B000682A712A7D2A882A9B2AA32AAF2A8316B2
:1004C000FC3090070530FF3E8312031D632AB72AD4
:1004D0008316043090070530FF3E8312031D6C2AFB
:1004E000B72A831610088312AB001F30A90004300E
:1004F000FF3E031D782A0000B72A0030AB001F30F2
:10050000A9000430FF3E031D822A862A0000B72A74
:100510000030AB0030302802031C942A0330FF3E29
:10052000031D8F2A0000982A2808E222AB00A80A9F
:100530001F30A900B72A0030A8000530FF3E031D78
:100540009E2A0000B72A2708AB001F30A900003000
:10055000A7000430FF3E031DAA2A0000B72A270A7D
:10056000031DA70A0530FF3E031DB32AB72AB82A88
:10057000B92AE02A0030AC0003302E05B100310862
:10058000213E84002A08800031083023B1002E1D4E
:10059000CC2A3108A504CF2AFF303106A505083042
:1005A000FF3E031DD02A0000E02A0030AC000F30CF
:1005B0002A05A5000E30FF3E031DDB2A0000E02ABD
:1005C00083120034840003308A000408003E820055
:1005D000000000000000000000000000000000001B
:1005E000000000000000000000000000000000000B
:1005F00000000000000000000000000000000000FB
:10060000013400340F340434003400340034003436
:10061000003400340034003400340034003400343A
:10062000003400340034003400340034003400342A
:10063000073453346534723476346F34343445348B
:100640000F344734723461346D346C34693463343C
:1006500068342634423465346E3473346F346E3407
:10066000840003308A000408363E820001340234DC
:040670000434083412
:02400E001E3161
:00000001FF
